:020000040800F2
:10000000D0120020D10800080507000807070008E3
:100010000B0700080F070008130700080000000086
:1000200000000000000000000000000017070008AA
:1000300019070008000000001B0700081D07000842
:10004000EB080008EB080008EB080008EB080008C4
:10005000EB080008EB080008EB080008EB080008B4
:10006000EB080008EB080008EB080008EB080008A4
:10007000EB080008EB080008EB080008EB08000894
:10008000EB080008EB080008EB080008EB08000884
:10009000EB080008EB080008EB080008EB08000874
:1000A000EB080008EB080008EB080008EB08000864
:1000B000EB080008EB080008EB080008EB08000854
:1000C000EB080008EB080008EB080008EB08000844
:1000D000EB080008EB080008EB080008232C0008D8
:1000E000EB080008EB080008EB080008EB08000824
:1000F000EB080008EB080008EB080008EB08000814
:10010000EB080008EB080008EB080008EB08000803
:10011000EB080008EB080008EB080008EB080008F3
:10012000EB080008EB080008EB08000803050008CE
:10013000DFF80CD002F074FE0048004765010008AB
:10014000D0120020EFF30980704780F309887047D0
:10015000EFF30880704780F30888704740BA704713
:10016000C0BA70471CB5002416A103C9CDE900012F
:100170004FF000601549086000F02CF802F090FD87
:1001800002F025FE4FF4E13000F0EEF801201049B6
:10019000086015E002F025FD012801D1012406E0E8
:1001A00002F056FC012801D1022400E00024012CB9
:1001B00002D102F0FEFC03E0022C01D102F0D2FCDD
:1001C000E8E700000301050A035C370008ED00E0E2
:1001D0008481224210B5042000F0DCFB2E48006828
:1001E00000EB400080002D49B0FBF1F02C49087075
:1001F0000846007800EB4001C1EBC0104FF6FF71DC
:1002000001EAC0002749088010BD0146244A12783F
:100210004A434FF0E0235A6100229A611A4612695C
:1002200042F001021A6100BF4FF0E022106910F0A5
:10023000010F02D010F4803FF6D04FF0E022126997
:1002400022F001024FF0E0231A6100229A61704708
:100250000146144A12884A434FF0E0235A610022B3
:100260009A611A46126942F001021A6100BF4FF00A
:10027000E022106910F0010F02D010F4803FF6D098
:100280004FF0E022126922F001024FF0E0231A61E0
:1002900000229A617047000004000020001BB70094
:1002A000000000200200002010B590B0044601219B
:1002B000880300F0A3FE0121084600F092FE0C9492
:1002C0000020ADF83400ADF83600ADF83800ADF8D8
:1002D0003C000C20ADF83A000CA9204801F0C3F80E
:1002E00001211E4801F04BF91D4801F07DFA1B4821
:1002F000001D01901B480290002003906420049090
:100300000020059080200690002007900890202073
:10031000099000020A9000200B9001A9104801F0FA
:1003200005FB012240210D4801F05AF901210C483A
:1003300001F027FB10B010BD10B5044600BF4021EE
:10034000064801F0F7F90028F9D04021034801F0F0
:10035000FEF92146014801F07FF910BD0038014047
:10036000580002404400002010B586B00446012128
:10037000682000F043FE0121880400F04CFE744820
:1003800001F02EF8734801F02FFA0420ADF81400A4
:1003900010208DF8170003208DF8160005A96E486F
:1003A00000F076FB4FF48060ADF8140018208DF853
:1003B000170005A9694800F06BFB4FF40060ADF829
:1003C000140004208DF8170005A9644800F060FBB4
:1003D00001940020ADF80800ADF80A00ADF80C005B
:1003E000ADF810000C20ADF80E0001A9584801F03E
:1003F0003AF827208DF8000001208DF80100022036
:100400008DF8020001208DF80300684600F077FAAD
:10041000012240F225514E4801F0BDF801214C481F
:1004200001F0ADF800204E49086006B010BD30B5AF
:100430008DB005460C464748143801F0D5F94448BC
:10044000001D029003951020049005940020069052
:10045000802007900020089009900A904FF40050E7
:100460000B9000200C9002A93A48143801F05EFA73
:1004700001228021364801F0B3F8012202213948D7
:1004800001F08BFA3B208DF8040002208DF8050066
:1004900001208DF806008DF8070001A800F02FFA62
:1004A0000DB030BD70B505460E4601202C490860E0
:1004B0004FF000040CE000BF4021254801F03AF95C
:1004C0000028F9D0295D224801F0C6F8601C84B2EA
:1004D000B442F0DB00BF40211D4801F02BF9002899
:1004E000F9D000201E49086070BD10B503460020F9
:1004F00000BF03E00C5C1C54441CE0B29042F9DBEA
:1005000010BD10B5184801F06AFA002111481438DE
:1005100001F037FA4FF49670FFF777FE002010498C
:10052000086010BD70B5044601200D4908602046E2
:1005300002F06EFCC5B229462046FFF7B3FF01204A
:10054000FFF786FE00200949C1F8880170BD000050
:10055000004800403000024000180140000C0140FB
:100560008801234258040240000002100000234288
:1005700000B585B00020ADF800004FF48270ADF8F2
:1005800002000020ADF80400ADF80600ADF8080048
:100590004FF40070ADF80A000020ADF80C00ADF883
:1005A0000E000720ADF810006946534800F0B8FD72
:1005B0000121514800F059FE05B000BD70B5054657
:1005C0000E46002405E0601CC4B2C82C01DD0020EA
:1005D00070BD0221284600F0CCFE0028F3D0314641
:1005E000284600F073FE002405E0601CC4B2C82C4D
:1005F00001DD0020ECE70121284600F0BAFE0028CA
:10060000F3D0284600F064FEC0B2E1E770B50546BD
:10061000002405E0601CC4B2C82C01DD002070BDC0
:100620000221364800F0A5FE0028F3D029463348C1
:1006300000F04CFE002405E0601CC4B2C82C01DDB3
:100640000020ECE701212D4800F093FE0028F3D0B4
:100650002A4800F03DFEC0B2E1E770B5054600242F
:1006600005E0601CC4B2C82C01DD002070BD022171
:10067000214800F07EFE0028F3D029461E4800F0F5
:1006800025FE002405E0601CC4B2C82C01DD00205A
:10069000ECE70121184800F06CFE0028F3D0164862
:1006A00000F016FEC0B2E1E770B50546002405E093
:1006B000601CC4B2C82C01DD002070BD02211048AE
:1006C00000F057FE0028F3D029460D4800F0FEFD4B
:1006D000002405E0601CC4B2FF2C01DD0020ECE723
:1006E0000121074800F045FE0028F3D0044800F03F
:1006F000EFFDC0B2E1E70000003C004000300140E7
:1007000000380040704700BFFEE700BFFEE700BFB3
:10071000FEE700BFFEE77047704770477047000074
:100720000CB50020019000905E48006840F48030D5
:100730005C49086000BF5B48006800F4003000902E
:100740000198401C0190009818B90198B0F5A06F6D
:10075000F1D15448006810F4003F02D0012000900D
:1007600001E0002000900098012828D14E48006840
:1007700040F010004C4908600846006820F0030073
:100780000860084600680860464840684549486077
:100790000846406848600846406848600846406827
:1007A00020F0030048600846406840F001004860BF
:1007B00000BF3C48406800F00C000428F9D10CBD93
:1007C00010B5FFF7ADFF10BD10B53648006840F01A
:1007D00001003449086008464068344908403149FE
:1007E000486008460068324908402E4908600846BB
:1007F000006820F4802008600846406820F4FE006D
:1008000048604FF41F008860FFF7DAFF4FF0006088
:100810002849086010BD10B5002100200022214B9E
:100820005B6803F00C0121B1042906D0082928D106
:1008300007E0214B214C236027E0214B1F4C236014
:1008400023E0184B5B6803F47010164B5B6803F4ED
:100850008032022303EB904022B91A4B4343174CDA
:1008600023600DE00F4B5B6813F4003F04D0164B80
:100870004343124C236003E0114B43430F4C23606E
:1008800003E00D4B0D4C236000BF00BF054B5B68C0
:10089000C3F303130D4CE15C084B1B68CB40074CC2
:1008A000236010BD00100240002002400000FFF84D
:1008B000FFFFF6FE08ED00E000127A0004000020C1
:1008C000001BB70000093D00808D5B000800002080
:1008D0000648804706480047FEE7FEE7FEE7FEE7DA
:1008E000FEE7FEE7FEE7FEE7FEE7FEE7C9070008D2
:1008F0003101000831490143314A1160704770B538
:10090000002100230F22C4780CB32D4C246804F47A
:10091000E064C4F5E064210AC1F10403CA404478EC
:1009200004FA03F18478144021430901254C067828
:10093000A155047804F01F050124AC4005786D1121
:100940004FF0E02606EB8505C5F8004109E0047884
:1009500004F01F050124AC401B4D0678761145F8C4
:10096000264070BD194A0A400243154B1B1F1A60EE
:10097000704739B1124A121D12680243104B1B1DF9
:100980001A6006E00E4A121D126882430C4B1B1DB2
:100990001A607047042808D14FF0E021096941F03E
:1009A00004014FF0E022116107E04FF0E0210969F6
:1009B00021F004014FF0E022116170470000FA05B8
:1009C0000CED00E000E400E080E100E080FFFF1FAC
:1009D00010B50446CA48844208D10121042000F021
:1009E00027FB0021042000F023FB46E0C548844299
:1009F00008D10121082000F01BFB0021082000F095
:100A000017FB3AE0C048844208D10121102000F0D1
:100A10000FFB0021102000F00BFB2EE0BB488442AE
:100A200008D10121202000F003FB0021202000F04C
:100A3000FFFA22E0B648844208D10121402000F0AC
:100A4000F7FA0021402000F0F3FA16E0B1488442A2
:100A500008D10121802000F0EBFA0021802000F075
:100A6000E7FA0AE0AC48844207D10121801500F082
:100A7000DFFA0021A01500F0DBFA10BD10B501214E
:100A8000084600F0D5FA0021012000F0D1FA10BD8F
:100A90002DE9F04102460025002600200023002415
:100AA000002791F803C00CF00F0591F803C01CF06B
:100AB000100F03D091F802C04CEA050591F800C070
:100AC000BCF1000F31D0146800202BE04FF0010C76
:100AD0000CFA00F3B1F800C00CEA03069E4220D1E4
:100AE00083004FF00F0C0CFA03F7BC4305FA03FC2C
:100AF0004CEA040491F803C0BCF1280F06D14FF072
:100B0000010C0CFA00FCC2F814C00AE091F803C012
:100B1000BCF1480F05D14FF0010C0CFA00FCC2F8F3
:100B200010C0401C0828D1D31460B1F800C0BCF13B
:100B3000FF0F34DD546800202EE000F1080C4FF068
:100B4000010808FA0CF3B1F800C00CEA03069E4253
:100B500021D183004FF00F0C0CFA03F7BC4305FAC8
:100B600003FC4CEA040491F803C0BCF1280F05D142
:100B700000F1080C08FA0CF8C2F8148091F803C0D0
:100B8000BCF1480F07D100F1080C4FF0010808FA3A
:100B90000CF8C2F81080401C0828CED35460BDE881
:100BA000F0814FF6FF710180022181700421C17034
:100BB00070470246002093680B4201D0012000E0FC
:100BC000002070470146886880B2704702460020C6
:100BD000D3680B4201D0012000E00020704701469D
:100BE000C86880B2704701617047416170470AB1BF
:100BF000016100E041617047C16070474FF480328D
:100C00000A4382618161826182698269704702461A
:100C10000020424B18684FF68073184040EA0210DB
:100C200008433E4B186070473D49C8617047F0B5B6
:100C30000A46002300240021002500F00046B6F1FA
:100C4000004F02D1354EF16901E0344E7168C0F3B6
:100C5000034583B200F44016B6F5401F08D121F0D9
:100C600070612E4E766826F070662C4F7E6012E022
:100C700000F48016B6F5801F06D1032606FA05F4A7
:100C8000A14341F0706106E0460D360103FA06F615
:100C9000B14341F0706122B1460D360103FA06F608
:100CA000314300F00046B6F1004F02D11B4EF16116
:100CB00001E01A4E7160F0BD30B500228B071C0FA9
:100CC0000F2303FA04F2154B08338C1053F8243029
:100CD0009343124C08348D1044F8253023468C1071
:100CE00053F824308C07240F00FA04F423430B4CF0
:100CF00008348D1044F8253030BD0A49086070472B
:100D000000080140000C01400010014000140140A7
:100D100000180140001C014000200140000001407B
:100D200000002042DC002042DD48006840F0010065
:100D3000DB49086008464068DA490840D8494860FD
:100D400008460068D8490840D54908600846006848
:100D500020F4802008600846406820F4FE004860C7
:100D60004FF41F0088607047CD49096821F4803135
:100D7000CB4A11601146096821F480211160B0F559
:100D8000803F03D0B0F5802F0ED106E0C44909683A
:100D900041F48031C24A116007E0C149096841F459
:100DA000A021BF4A116000E000BF00BF704710B52E
:100DB00001460022002300204A11012A02D1B84C2A
:100DC000236806E0022A02D1B54C236A01E0B44C44
:100DD000636A01F01F02012494401C4201D00120EB
:100DE00000E0002010BD38B5002000900024002550
:100DF00000BF3120FFF7DBFF05460098401C009044
:100E00000098B0F5A06F01D0002DF2D03120FFF78F
:100E1000CEFF08B1012400E00024204638BD014681
:100E200000209F4A106820F0F80040EAC1001060DE
:100E300070479E490860704702460020984B5868EA
:100E400020F47C1042EA01031843954B5860704728
:100E500096490866704701460020914A506820F084
:100E600003000843506070478D48406800F00C0054
:100E70007047014600208A4A506820F0F00008437D
:100E80005060704701460020854A506820F4E060B9
:100E900008435060704701460020814A506820F4A2
:100EA000605040EAC1005060704729B17C4A527AD4
:100EB00002437B4B5A7204E0794A527A8243784B60
:100EC0005A7270477A490860704701460020744A98
:100ED000506820F440400843506070470021754A34
:100EE00011706F4A82F82010012802D0042808D11E
:100EF00003E001216F4A117004E005216D4A117071
:100F000000E000BF00BF70476B490860704764494C
:100F1000096A0143624A11627047674944390860AF
:100F2000704730B500210022002400235C4D6D681D
:100F300005F00C0121B1042905D0082923D105E0D1
:100F40005E4D056022E05E4D05601FE0544D6D680A
:100F500005F47012524D6D6805F48034022505EBDE
:100F600092421CB9574D554305600BE04C4D6D68DE
:100F700015F4003F03D0544D5543056002E0504D39
:100F80005543056002E04D4D056000BF00BF444D74
:100F90006D6805F0F00109094C4D6B5C0568DD409A
:100FA00045603F4D6D6805F4E061090A474D6B5C93
:100FB0004568DD4085603A4D6D6805F46051C90AA9
:100FC000424D6B5C4568DD40C560354D6D6805F48C
:100FD0004041890B3E4D6B5CC568B5FBF3F505617F
:100FE00030BD29B12E4A526902432D4B5A6104E0AB
:100FF0002B4A526982432A4B5A61704729B1284AC9
:1010000092690243264B9A6104E0254A9269824321
:10101000234B9A61704729B1214AD2690243204B80
:10102000DA6104E01E4AD26982431D4BDA617047DF
:1010300029B11B4AD2680243194BDA6004E0184A0E
:10104000D2688243164BDA60704729B1144A12699C
:101050000243134B1A6104E0114A12698243104B98
:101060001A61704714494039086070470F49C864D5
:1010700070470B49C87170470948406A40F080705A
:1010800007494862704701460020054A92680A42B3
:1010900001D0012000E000207047014988727047AC
:1010A000001002400000FFF8FFFFF6FE0000424281
:1010B000D8004242201002408004424200127A00CE
:1010C000001BB70000093D00808D5B001800002068
:1010D0002800002010B50446BE48844208D10121F2
:1010E0008014FFF7A5FF0021A014FFF7A1FF16E071
:1010F000B948844208D101210014FFF7A6FF00215E
:101100002014FFF7A2FF0AE0B448844207D101216E
:10111000C013FFF79AFF0021E013FFF796FF10BD01
:1011200010B50022028802F441520B884C882343F8
:101130008C882343CC8823430C8923434C89234345
:101140008C892343CC8923431A430280838B4FF23B
:10115000FF74234083830B8A038210BD2DE9F04F77
:1011600085B005460C464FF0000902274FF00008F5
:101170004FF0010B0026B246A88B4FF24001084009
:10118000A88302202884B5F81C90A068022801D109
:1011900000BF38E0A08810B94FF0010B01E04FF01C
:1011A000020B8D48854200D100E000BF6846FFF782
:1011B000B8FEDDF800A0E088B0F5007F0AD14FEA64
:1011C0001A2000EB80004000A168B0FBF1F0401D48
:1011D00086B20BE04FEA4B10BAFBF0F000EB800058
:1011E0004000A168B0FBF1F0401D86B20A20B6FBBA
:1011F000F0F606F00108A6EB0800C0F34F074FF623
:10120000FF7000EA0828022F01DBFF2F02DD022712
:101210004FF00008E08840EA080038432884A0889E
:10122000A1890843618808432188084340F400608D
:1012300040EA0909A5F81C9005B0BDE8F08F00212F
:10124000018041808180C180018141818181C18192
:101250000721018270470021018041808180C18087
:101260000221816000218181704721B1028842F012
:101270004002028004E002884FF6BF731A400280E9
:10128000704721B1828B42F48062828304E0828BBA
:101290004FF6FF331A408283704730B50024002395
:1012A0000C110125A540ABB21AB185881D4385807C
:1012B00002E085889D43858030BD1AB183880B4349
:1012C000838002E083888B438380704781817047ED
:1012D000014688897047A1F57E42FF3A04D0028812
:1012E00042F48072028004E002884FF6FF631A40E5
:1012F0000280704721B1828842F00402828004E0BB
:1013000082884FF6FB731A408280704702884FF242
:10131000FF731A40028002880A43028070470188E6
:1013200041F480510180704721B1028842F400529B
:10133000028004E002884DF6FF731A400280704775
:1013400002460020012901D0108B00E0908A7047EE
:101350000146088A7047B1F5804F04D1028842F4F3
:101360008042028004E002884BF6FF731A4002803C
:1013700070470246002013890B4201D0012000E093
:1013800000207047CA4302817047F0B50246002032
:1013900000240023002501F00F070126BE40B4B24F
:1013A0000B1101269E40B3B2968806EA0305168902
:1013B000264202D00DB1012000E00020F0BD10B5A2
:1013C000002201F00F040123A3409AB2D34303810A
:1013D00010BD00000030014000380040003C0040DB
:1013E00010B50446FB48844209D101218803FFF768
:1013F0001FFE00214FF48040FFF71AFE32E0F6484E
:10140000844209D101214804FFF71FFE00214FF457
:101410000030FFF71AFE25E0F048844209D101218F
:101420008804FFF712FE00214FF48020FFF70DFE25
:1014300018E0EB48844209D10121C804FFF705FEFA
:1014400000214FF40020FFF700FE0BE0E548844246
:1014500008D101210805FFF7F8FD00214FF48010A5
:10146000FFF7F3FD10BD2DE9F04786B005460E46A7
:101470000024A24600BFA1460027B08900B100BFEA
:101480002F462C8A4CF6FF700440F08804432C82CF
:10149000AC894EF6F3100440B08831890843718955
:1014A00008430443AC81AC8A4FF6FF400440B08946
:1014B0000443AC8201A8FFF734FDC648874202D13D
:1014C000DDF810A001E0DDF80CA0A88910F4004FB1
:1014D00008D00AEBCA0000EB0A1031684900B0FBE3
:1014E000F1F807E00AEBCA0000EB0A103168890046
:1014F000B0FBF1F86420B8FBF0F00401200964218E
:1015000001FB1089A88910F4004F08D0322000EBAD
:10151000C900B0FBF1F000F00700044308E03220FE
:1015200000EB09106421B0FBF1F000F00F00044360
:101530002C8106B0BDE8F0874FF416510160002100
:101540008180C18001810C2141810021818170470E
:1015500010B502460020108A4FF2FF0318400B8896
:101560004C8823438C882343CC8823431843108220
:1015700010BD0021018041808180C180704721B170
:10158000828942F40052828104E082894DF6FF7321
:101590001A4082817047F0B50346002400260025DA
:1015A0000020A1F510676A3F00D100BF1846C1F3C3
:1015B000421401F01F06012707FA06F5012C01D19C
:1015C0000C3004E0022C01D1103000E014301AB1CC
:1015D00007682F43076002E00768AF430760F0BD6C
:1015E0001AB1838A0B43838202E0838A8B4383820E
:1015F0007047028A4FF6F0731A400282028A0A4349
:101600000282704782894FF2FF731A408281828979
:101610000A438281704721B1828942F002028281AD
:1016200004E082894FF6FD731A4082817047028A76
:101630004FF6DF731A400282028A0A430282704721
:1016400021B1028A42F48042028204E0028A4BF60F
:10165000FF731A4002827047C1F30802828070470C
:1016600001468888C0F308007047818941F0010174
:1016700081817047028BD2B20283028B42EA01223F
:1016800002837047028B02F47F420283028B0A437B
:101690000283704721B1828A42F02002828204E0F4
:1016A000828A4FF6DF731A408282704721B1828AA4
:1016B00042F01002828204E0828A4FF6EF731A40F1
:1016C0008282704721B1828A42F00802828204E05D
:1016D000828A4FF6F7731A408282704721B182895D
:1016E00042F40042828103E08289C2F30E028281C9
:1016F000704721B1828A42F40062828204E0828AC9
:101700004FF2FF731A4082827047828A4FF6FB7352
:101710001A408282828A0A438282704721B1828A79
:1017200042F00202828204E0828A4FF6FD731A4080
:101730008282704702460020B1F5007F00D100BFD1
:1017400013880B4201D0012000E00020704701F413
:101750000072B2F5007F00D100BFCA43028070471B
:1017600070B502460024002300250020A1F5106674
:101770006A3E00D100BFC1F3421501F01F030126EC
:1017800006FA03F3012D02D19689334006E0022DBB
:1017900002D1168A334001E0968A33400C120126AA
:1017A00006FA04F41688344013B10CB1012000E0AD
:1017B000002070BD10B500220023A1F510646A3C22
:1017C00000D100BF0A1201249440A3B2DC4304807C
:1017D00010BD0000003801400044004000480040B7
:1017E000004C00400050004001684FF6FE7211406E
:1017F00001600021016041608160C1608C498842C4
:1018000008D18B490839496841F00F01884A083AE4
:1018100051608AE086491431884208D184490839E8
:10182000496841F0F001824A083A51607DE0804900
:101830002831884208D17E490839496841F47061ED
:101840007B4A083A516070E079493C31884208D1BE
:1018500077490839496841F47041754A083A51603E
:1018600063E073495031884208D1714908394968A9
:1018700041F470216E4A083A516056E06C49643177
:10188000884208D16A490839496841F47001684AB8
:10189000083A516049E066497831884208D1644984
:1018A0000839496841F07061614A083A51603CE08A
:1018B0006049884206D1011F096841F00F01021FEB
:1018C000116032E05B491431884208D15949091F3F
:1018D000096841F0F001574A121F116025E055498F
:1018E0002831884208D15349091F096841F47061C1
:1018F000504A121F116018E04E493C31884208D10D
:101900004C49091F096841F470414A4A121F11608D
:101910000BE048495031884207D14649091F096800
:1019200041F47021434A121F1160704710B5002224
:10193000026847F6F0739A430C6A8B6823430C697C
:1019400023434C6923438C692343CC6923434C6A6A
:1019500023438C6A23431A430260CB6843600B68BD
:1019600083604B68C36010BD0021016041608160ED
:10197000C160016141618161C16101624162816255
:10198000704721B1026842F00102026004E002687F
:101990004FF6FE731A40026070471AB103680B439A
:1019A000036002E003688B43036070474160704747
:1019B0000146486880B2704701460020002211F0BD
:1019C000805F03D01B4B083B1A6802E0184B083BB2
:1019D0001A680A4201D0012000E00020704710F090
:1019E000805F03D01349091F086002E010490839DD
:1019F0004860704701460020002211F0805F03D04C
:101A00000C4B083B1A6802E0094B083B1A680A4273
:101A100001D0012000E00020704710F0805F03D06B
:101A20000449091F086002E001490839486070470D
:101A3000080002400804024001460020FE4A1068E7
:101A400000F03800084310607047FB49096821F036
:101A50000801F94A11601146096801431160704795
:101A6000F549096821F01001F34A1160114609682F
:101A7000014311607047F148EF494860F048486001
:101A80007047EE48EC494860ED4848607047EA48C6
:101A9000006940F08000E84908617047E648006945
:101AA00040F08000E449086170470420E249C968B9
:101AB00011F0010F01D001200EE0DF49C96811F0DB
:101AC000040F01D0022007E0DB49C96811F0100FB4
:101AD00001D0032000E00420704700B50246042333
:101AE000FFF7E3FF034603E0FFF7DFFF0346521E65
:101AF000012B01D1002AF7D102B90523184600BDF8
:101B000030B5044604254FF43020FFF7E6FF0546C4
:101B1000042D17D1C848006940F00200C649086189
:101B200008464461006940F0400008614FF43020ED
:101B3000FFF7D3FF0546C048006941F6FD71084034
:101B4000BD490861284630BD10B504244FF430204B
:101B5000FFF7C3FF0446042C16D1B748006940F0D4
:101B60000400B54908610846006940F0400008617A
:101B70004FF43020FFF7B1FF0446AF48006941F64B
:101B8000FB710840AC490861204610BD00B5024613
:101B90000423FFF78AFF034603E0FFF786FF0346AF
:101BA000521E012B01D1002AF7D102B90523184694
:101BB00000BD10B504244FF43020FFF7E7FF0446C2
:101BC000042C16D19C48006940F004009A49086131
:101BD0000846006940F0400008614FF43020FFF7EC
:101BE000D5FF04469448006941F6FB7108409249CC
:101BF0000861204610BD00208F49C96911F0020F0D
:101C000001D0012000E00020704730B5A525042454
:101C1000FFF7F1FF00B100254FF43020FFF75DFF23
:101C20000446042C3AD185488349886084488860FA
:101C30000846006940F0200008610846006940F04D
:101C4000400008614FF43020FFF747FF0446042CA2
:101C50001BD17948006941F6DF7108407649086177
:101C60000846006940F01000086176480580E002EF
:101C7000FFF733FF0446052C10D06F48006941F68A
:101C8000EF7108406C49086108E0052C06D06A48ED
:101C9000006941F6EF71084067490861204630BD90
:101CA00078B506460C46042500200090E802FFF7B0
:101CB00014FF0546042D24D15F48006940F001005F
:101CC0005D4908613480E802FFF707FF0546042DEF
:101CD00010D1B01C0090200C00990880E802FFF79A
:101CE000FCFE05465448006941F6FE710840524921
:101CF000086106E05048006941F6FE7108404E490F
:101D00000861284678BD70B504460D460426F002E9
:101D1000FFF7E3FE0646042E11D14748006940F064
:101D20000100454908612580F002FFF7D6FE06460E
:101D30004148006941F6FE7108403F49086130465C
:101D400070BD70B505460E460424E002FFF7C5FEDF
:101D50000446042C17D139483749886038488860D0
:101D60000846006940F0100008612E80E002FFF78D
:101D7000B4FE0446052C06D02F48006941F6EF71E9
:101D800008402D490861204670BD2DE9F043044606
:101D90004FF6FF763746B046B1460425E443E6B237
:101DA000C4F30727C4F307484FEA1469E802FFF7B2
:101DB00094FE0546042D49D120481F4988602048DB
:101DC00088600846006940F010000861FF2E06D0C8
:101DD0001C4808300680E802FFF77FFE0546042D08
:101DE00008D1FF2F06D017480A300780E802FFF716
:101DF00074FE0546042D0AD1B8F1FF0F07D0114833
:101E00000C30A0F80080E802FFF767FE0546042DBD
:101E10000AD1B9F1FF0F07D00A480E30A0F80090A0
:101E2000E802FFF75AFE0546052D0FD0024800696B
:101E300041F6EF71084007E00020024023016745AA
:101E4000AB89EFCD00F8FF1F664908612846BDE861
:101E5000F08330B5054604244FF43020FFF73DFEF3
:101E60000446042C41D160485E4988605F48886020
:101E70000846006940F0200008610846006940F00B
:101E8000400008614FF43020FFF727FE0446042C81
:101E900022D15448006941F6DF7108405149086178
:101EA0000846006940F0100008611DB1002050494B
:101EB000088002E0A5204E4908804FF43020FFF74B
:101EC0000CFE0446052C10D04648006941F6EF711F
:101ED00008404449086108E0052C06D041480069E3
:101EE00041F6DF7108403F490861204630BDF0B53A
:101EF00005460E46174604243B483A4988603B484D
:101F00008860E002FFF7E9FD0446042C19D135484A
:101F1000006940F010003349086147F0F800304391
:101F200028433349891C0880E002FFF7D6FD0446A8
:101F3000052C06D02B48006941F6EF71084029496D
:101F400008612046F0BD2748C069800870472548D1
:101F5000006A704700202349096811F0200F01D062
:101F6000012000E00020704729B11E4A1269024397
:101F70001C4B1A6104E01B4A12698243194B1A6117
:101F8000704701460020012908D1164AD26912F093
:101F9000010F01D0012008E0002006E0114AD268BC
:101FA0000A4201D0012000E0002070470D49C860BE
:101FB000704704200B49C96811F0010F01D00120BE
:101FC0000EE00849C96811F0040F01D0022007E0B3
:101FD0000449C96811F0100F01D0032000E004206B
:101FE000704700000020024023016745AB89EFCD18
:101FF00000F8FF1F08B54FF48070ADF80000102006
:102000008DF8030003208DF802006946FE48FEF7B4
:102010003FFD0020FD49086008BD08B54FF4806011
:10202000ADF8000010208DF8030003208DF80200A9
:102030006946F748FEF72CFD4FF40060ADF800004C
:1020400010208DF8030003208DF802006946F04847
:10205000FEF71EFD4FF48050ADF8000010208DF803
:10206000030003208DF802006946E948FEF710FDE1
:1020700008BD08B54020ADF8000010208DF8030021
:1020800003208DF802006946E248FEF701FD4FF497
:102090000040ADF8000010208DF8030003208DF8FB
:1020A00002006946DA48FEF7F3FC08BD08B538209F
:1020B000ADF8000018208DF8030003208DF8020011
:1020C0006946D548FEF7E4FC8020ADF800001020FA
:1020D0008DF8030003208DF802006946CE48FEF714
:1020E000D7FC8021CC48FEF77EFD8020ADF80000B3
:1020F00010208DF8030003208DF802006946C448C3
:10210000FEF7C6FC8021C248FEF76DFD08BD08B58C
:102110000820ADF8000010208DF8030003208DF892
:1021200002006946BD48FEF7B3FC0020BC490860C8
:1021300008BD08B50820ADF8000000208DF80300A8
:1021400003208DF802006946B448FEF7A1FC08BDE3
:1021500008B50120ADF8000010208DF80300032021
:102160008DF802006946AD48FEF792FC0220ADF8FA
:10217000000010208DF8030003208DF8020069464E
:10218000A648FEF785FC4FF48070ADF800001020E3
:102190008DF8030003208DF8020069469E48FEF783
:1021A00077FC4FF40070ADF8000010208DF80300AC
:1021B00003208DF8020069469748FEF769FC01216B
:1021C0009648FEF710FD08BD08B50120ADF80000E7
:1021D00028208DF8030003208DF8020069468F48FF
:1021E000FEF756FC0220ADF8000028208DF8030011
:1021F00003208DF8020069468848FEF749FC4FF439
:102200008070ADF8000028208DF8030003208DF8C1
:10221000020069468048FEF73BFC4FF40070ADF8C1
:10222000000028208DF8030003208DF80200694685
:102230007948FEF72DFC08BD08B501210420FEF702
:10224000DDFEFF20ADF8000010208DF80300032014
:102250008DF8020069466C48FEF71AFC012108203F
:10226000FEF7CCFE4FF44050ADF8000028208DF86A
:10227000030003208DF8020069466748FEF708FC5A
:102280004FF44040ADF8000010208DF8030003200B
:102290008DF8020069466048FEF7FAFB01214020F4
:1022A000FEF7ACFE4020ADF8000010208DF80300D2
:1022B00003208DF8020069465848FEF7E9FB00202C
:1022C000584908605849C1F8B80158490860584948
:1022D000086001F10401086001F10401086001F1E6
:1022E0000401086001F10401086001F104010860C3
:1022F00001F10401086001F10401086008BD08B59E
:1023000001210420FEF77AFEFF20ADF80000002036
:102310008DF8030003208DF8020069463A48FEF765
:10232000B7FB01210820FEF769FE4FF44050ADF8DD
:10233000000000208DF8030003208DF8020069469C
:102340003548FEF7A5FB4FF44040ADF800000020F3
:102350008DF8030003208DF8020069462E48FEF731
:1023600097FB01214020FEF749FE4020ADF8000018
:1023700000208DF8030003208DF8020069462748ED
:10238000FEF786FB08BD08B50220ADF8000000206E
:102390008DF8030069461F48FEF77AFB0120ADF86F
:1023A000000000208DF8030069461A48FEF770FB14
:1023B00008BD08B50220ADF8000000208DF803002C
:1023C00069461448FEF764FB08BD08B50120ADF866
:1023D000000000208DF8030069460E48FEF758FB08
:1023E00008BD08B58020ADF8000028208DF8030056
:1023F00069460848FEF74CFB4FF48070ADF80000CA
:102400006946044816E0000000080140A00121428E
:102410000014014000100140000C01400018014070
:102420008C0123429801234200802142BC81214239
:1024300080012142FEF72CFB4FF40070ADF8000044
:102440006946FE48FEF724FB08BD08B50220ADF83A
:10245000000010208DF8030003208DF8020069466B
:10246000F748FEF715FB0020F649086008BD08B5DF
:102470004FF40070ADF8000018208DF80300694695
:10248000F148FEF705FB4FF48060ADF80000042032
:102490008DF803006946EC48FEF7FAFA08BD08B566
:1024A0004FF40070ADF8000000208DF8030069467D
:1024B000E548FEF7EDFA4FF48060ADF8000000202B
:1024C0008DF803006946E048FEF7E2FA4FF48070A9
:1024D000ADF8000000208DF8030003208DF8020005
:1024E0006946D948FEF7D4FA08BD08B54FF4005044
:1024F000ADF8000010208DF8030003208DF80200D5
:102500006946D248FEF7C4FA4FF48040ADF80000A7
:1025100010208DF8030003208DF802006946CB4897
:10252000FEF7B6FA4FF40060ADF8000028208DF8F1
:1025300003006946C548FEF7ABFA4FF40051C348A3
:10254000FEF751FB4FF48041C048FEF74CFB08BD3D
:1025500008B54FF40050ADF8000018208DF80300C6
:1025600003208DF802006946B548FEF791FA08BDD0
:1025700008B54FF40040ADF8000010208DF80300BE
:1025800003208DF802006946AD48FEF781FA4FF44A
:102590000041AB48FEF729FB08BD08B54FF40050D9
:1025A000ADF8000000208DF8030003208DF8020034
:1025B0006946A348FEF76CFA08BD08B54FF4004021
:1025C000ADF8000010208DF8030003208DF8020004
:1025D00069469D48FEF75CFA00209D49086008BDE9
:1025E00008B58020ADF8000010208DF8030003200E
:1025F0008DF8020069469548FEF74AFA0020954991
:10260000086008BD08B58020ADF8000010208DF8E6
:10261000030003208DF8020069468C48FEF738FA63
:1026200000208C49086008BD08B50220ADF8000004
:1026300010208DF8030003208DF8020069468048C1
:10264000FEF726FA00207F49086008BD08B54FF460
:102650008060ADF8000018208DF8030003208DF88D
:10266000020069467C48FEF713FA4FF40060ADF8AB
:10267000000004208DF8030003208DF80200694655
:102680007548FEF705FA4FF48070ADF80000102091
:102690008DF8030003208DF8020069466B48FEF7B1
:1026A000F7F901206D49086008BD08B58020ADF834
:1026B000000000208DF8030003208DF80200694619
:1026C0006248FEF7E5F94FF48060ADF800000020A5
:1026D0008DF8030003208DF8020069465E48FEF77E
:1026E000D7F94FF40060ADF8000000208DF803002A
:1026F00069465948FEF7CCF94FF48070ADF80000F8
:1027000000208DF8030003208DF8020069464F4831
:10271000FEF7BEF901205149086008BD08B5012047
:10272000ADF8000010208DF8030003208DF80200A2
:1027300069464948FEF7ACF94FF40060ADF8000077
:1027400010208DF8030003208DF8020069463F48F1
:10275000FEF79EF90020424908604249C1F8800115
:1027600008BD08B52020ADF8000010208DF803004A
:1027700003208DF8020069463048FEF789F90020F1
:102780003949086008BD08B54FF40060ADF8000095
:1027900010208DF8030003208DF8020069462B48B5
:1027A000FEF776F900202E49086008BD08B54FF401
:1027B0000060ADF8000004208DF8030003208DF8C0
:1027C000020069462048FEF763F908BD704708B566
:1027D0004FF2FF70ADF8000000208DF8030069464D
:1027E0001948FEF755F94FF6FF70ADF800000020CC
:1027F0008DF8030069461848FEF74AF94FF6F7705E
:10280000ADF8000000208DF8030069460B48FEF784
:102810003FF90820ADF8000004208DF80300694658
:102820000648FEF735F94FF6FF70ADF800000020BE
:102830008DF803006946024818E0000000100140CE
:102840000014014084812242000801400018014028
:10285000BC0121429C012342000C0140A001234203
:10286000AC0123420080214294012242FEF710F97C
:1028700047F6F770ADF8000000208DF803006946B8
:102880000148FEF705F908BD0018014070B504467F
:102890000D46002305E026782E706D1C641C5E1C1E
:1028A000F3B29342F7DB70BD0146088870472DE90B
:1028B000F04105460E461746002407E036F814108E
:1028C0002846FFF720FAAD1C601C84B2BC42F5DB41
:1028D000BDE8F08130B503460C461546002207E0FE
:1028E0001846FFF7E1FF24F812009B1C501C82B22F
:1028F000AA42F5DB30BD2DE9F04106460F461446ED
:10290000204604EBD0714910A4EB4101012905D107
:1029100004EBD0714910491C8DB203E0204604EB52
:10292000D0714D10FFF7A7F82A4631463846FFF719
:10293000BEFFFFF7ACF8BDE8F08110B5C6480068EF
:10294000002857D0C5480078002854DD00BFC34890
:102950000078401DC04909688842F8D8BF48C0784F
:10296000B8B900240DE0201DBC49085CBC49BD4A33
:1029700012688854BB480068401CBA490860601C53
:10298000C4B2B6480078A042EDDC0020B24908602D
:1029900013E0B248C07805280FD1B0480079B24999
:1029A0000870AE4840794870AC4880798870AB4870
:1029B000C079C8700020A8490860AA480068B0F52E
:1029C000006F0FD14FF40062A8480168A448FFF7D8
:1029D00092FFA648006800F50060A4490860002046
:1029E000A04908609D490978091D9C4A8818012161
:1029F000FDF758FD2BE098480068052827D1974837
:102A0000407820BB9548807808BB9448C07801285E
:102A10001DD192480079FF2819D19248008882B2CE
:102A2000924801688E48FFF766FF904800688D491C
:102A3000096808448D49086000208A49086001201F
:102A40008B49087001218548001DFDF72BFD10BD45
:102A500081480068002841D080480078854909787D
:102A6000884238D17C48006807282CD17B484078C0
:102A700080494978884222D1784880787D49897890
:102A800088421CD17548C0787A49C978884216D1E5
:102A90007248007977490979884210D16F484079A6
:102AA0007449497988420AD16C4880797149897999
:102AB000884204D100206849086001207047002046
:102AC000654908600AE064480068072806D90020C4
:102AD0006149086002E000205F4908600020EDE7DE
:102AE00010B5654CFEF7C7FF00BF04E02046FFF7B6
:102AF00007F804F5006461488442F7D3FEF7C7FF86
:102B000010BD70B505460024FEF7B5FF5C48FEF722
:102B1000F7FF10225B495A48FFF7C9FEFEF7B7FFDF
:102B200070BD10B50446206857490840B0F1005FF9
:102B300017D16068554908602068FDF70CFB72B634
:102B400000215348FEF71BFD0520FDF781FB002007
:102B5000504908604FF00A00FDF77AFB4B480068C7
:102B6000804710BD00BFFFF7BBFF00203A49086057
:102B70003C49086040483D49086000203C490870D5
:102B800007214548FDF78EFC12E001E0FFF7D5FE76
:102B9000374800780028F9D006E034480068FFF78D
:102BA000B0FF3548FFF7BDFF314800780128F4D069
:102BB000EBE710B572B600213548FEF7E0FC0520C2
:102BC000FDF746FB0020334908604FF00A00FDF78F
:102BD0003FFB002080F3108800BF2748FFF7A1FFCC
:102BE00010BD10B5FEF747FF10222C492448FFF70F
:102BF00071FEFEF74CFF00240AE0284830F814006C
:102C0000204931F81410884200D003E0601CC4B29F
:102C1000102CF2DB00BF0F2C01DD012010BD0020C5
:102C2000FCE710B540F225511948FEF799FD88B12F
:102C30001748FEF715FD0949074A126888540648E7
:102C40000068401C0449086008460068642801D3F5
:102C50000020086010BD0000380000207201002034
:102C6000420200203C000020300000202C00002008
:102C700034000020702E00080080000800000808C2
:102C800000780008782E00080000FE2F4000002089
:102C90000048004084812242622E0008A60A0020DB
:102CA00010B501217C20FEF7A9F901210846FEF7A5
:102CB000A5F9FFF77BFDFFF7F9F9FFF7C6FBFFF773
:102CC00026FA01204D490860FFF742FAFFF726FD7A
:102CD000FFF70BFCFFF73CFCFFF74AFCFFF781FB1B
:102CE000FFF76BFCFFF70BFBFFF77AFCFFF76EFDBE
:102CF00010BD08B501215020FEF780F903208DF8A2
:102D0000020048208DF803000120ADF8000069465C
:102D10003B48FDF7BDFE4FF40070ADF8000069467A
:102D20003848FDF7B5FE10208DF803000220ADF8FD
:102D3000000069463248FDF7ABFE4FF48060ADF805
:102D4000000069462F48FDF7A3FE4FF480612D482F
:102D5000FDF749FF02212A48FDF745FF01202A49D6
:102D6000086008BD10B501217C20FEF747F901215C
:102D70000846FEF743F9FFF7CAF901201F4908602A
:102D8000FFF7E6F9FFF7CAFCFFF7AFFBFFF729FBF8
:102D9000FFF71CFD10BD10B54FF48030FDF7E4FFC8
:102DA000FEF721F80446012C10D10020FEF761F84F
:102DB000A002FEF767F80020FEF76DF80120FEF78D
:102DC0004AF800BFFEF750F80428FBD110BD10B53B
:102DD0000121C803FEF71FF901210846FEF70EF98D
:102DE00001210A48FDF723FFFDF7C2FB10BD10B516
:102DF0004FF4E130FDF758FA10BD00008C0123427A
:102E000000100140001801409401224200023000ED
:102E1000421C10F8011B0029FBD1801A70470000EA
:102E2000064C074D06E0E06840F0010394E8070017
:102E300098471034AC42F6D3FDF77EF9982E00087F
:102E4000B82E000802E008C8121F08C1002AFAD1F3
:102E500070477047002001E001C1121F002AFBD11A
:102E600070470301AA55038D3E0301050A035C3731
:102E7000040255AA03C9FA00000011002200330021
:102E8000440055006600770088009900AA00BB0046
:102E9000CC00DD00EE00FF00B82E0008000000208E
:102EA00044000000442E0008FC2E000844000020CE
:102EB0008C120000542E000800000000001BB70018
:102EC00000000000000000000102030406070809DA
:102ED00000000000010203040102030406070809C0
:102EE00002040608000000000000000000000000CE
:0C2EF000000000000000000000000000D6
:0400000508000131BD
:00000001FF
